:1000000000001F308A00A02FF000030EF10004084A
:10001000F2000A08F3008A01831203130B1E1D2845
:100020008B1C1D28FF303506031D1A28B60A003028
:10003000B5001B28B50A8B103E28831603130C1C31
:100040003E28831203130C1C3E28B40B37280230C1
:10005000B4003508B7003608B800B501B601B003E2
:1000600000303006031D3728FF30B000B103AE0961
:100070000D308F0000308E000C103E2883120313C9
:1000800073088A0072088400710E8300F00E700EEF
:100090008312031309008316031303308600FF3015
:1000A0008500C730870083120313831603130730BC
:1000B0009F000730810050308B0001308C0083128C
:1000C000031338309000850186018701AF01FC21C0
:1000D000D421E621D421E021D4216E284C217321A2
:1000E000831603138B1783120313B501B6018A110C
:1000F0000A16122BFF30B0000330B100AF01003000
:10010000310603198712E6212030E9212030E92148
:100110002030E9213708BA00BC00B3003808B90024
:10012000BB00B20058213908BB003A08BC00582176
:100130003208BB003308BC00582182212030E9215D
:100140001030A7008D30A8008A110A1600238A11EA
:100150000A12E021051CB92887122E1CB12844215F
:100160007E281630A8008A110A1600238A110A1266
:100170007E28851EC7282E1CBF2844217E282730B4
:10018000A8008A110A1600238A110A127E28442127
:100190008518CE28871687152F14D42805197E2890
:1001A00087160716AF14D428E6212030E921203025
:1001B000E9212030E9213708BA00BC00B300380833
:1001C000B900BB00B20058213908BB003A08BC0096
:1001D00058213208BB003308BC005821822120304E
:1001E000E9211030A7008D30A8008A110A160023DB
:1001F0008A110A12E02105181729851900292629D4
:10020000051A03293429AF1C0D296B30A8008A1167
:100210000A1600238A110A12D4282F1CD4285A3017
:10022000A8008A110A1600238A110A12D42807127C
:1002300087111630A8008A110A1600238A110A12A3
:100240000430AD006C218712AF017A2807128711A4
:100250007C30A8008A110A1600238A110A12043081
:10026000AD006C21AF017A2887127C30A8008A117A
:100270000A1600238A110A120430AD006C210712FD
:1002800087118716AF017A284930A8008A110A160B
:1002900000238A110A1208000230B4000D308F00CA
:1002A00000308E00B501B70110148B158B170800B4
:1002B0003B08B9073C08BA070318B90A08006430BC
:1002C000AC000430AB00FA30AA00AA0B6529AB0BD6
:1002D0006329AC0B612908005F21AD0B6C29080074
:1002E0003E30A90008001E30A90008000E30A90009
:1002F00008000630A90008000230A90008000030FC
:10030000A9000800390EF038F500F507E23EF600C6
:10031000323EF80039080F39F607F607F807E93ECC
:10032000F700F707F7073A0E0F39F707F807F70D49
:10033000F80DF809F80D3A080F39F807F50D0730F0
:10034000F4000A30F807F703031CA229F707F603A5
:10035000031CA629F607F503031CAA29F507F403D5
:10036000031CAE297408303EA91EB729E92175087F
:10037000303E291EBC29E9217608303EA91DC1293D
:10038000E9217708303E291DC629E9217808303E49
:10039000A91C0800E9210800E6219030222208006B
:1003A000E021D0302222080001302222472A1330D7
:1003B000A100C030222247222030E921A10BDC29F4
:1003C000C0302222472A02302222472A80302222AD
:1003D000472AA00043220F3086052008F039860402
:1003E00086100615861586110F308605200EF03909
:1003F000860486158611080086110611861047228C
:100400000F3086053030860483160F3006058600CF
:10041000831286158611FC30A20004303522861521
:10042000861143228615861143220F30860520301F
:1004300086048615861128302222083022220C30AC
:1004400022220630A00043220F3086052008F03912
:10045000860486100611861586110F308605200E3B
:10046000F0398604861586110800A3000130A40027
:10047000A5000000A20B392AA30B392AA40B392AA4
:10048000A50B392A08001630A2000130352A9C300D
:10049000A2000F30352AFF3FFF3FFF3FFF3FFF3FE6
:1020000054346D346E34003452346F3474342034AC
:102010004E346F3472346D34003452346F3474344F
:10202000203449346E347634203400342034203463
:1020300041345234523445345434203455345234BB
:10204000473445344E34433445342034003443342B
:102050004C3445342034413420344D3441344E34F2
:102060004434523449344E34203420342034003443
:10207000563461347234693461347434653475347F
:1020800072342034613472347234653474342034E0
:1020900000342034203420342034203420342034C0
:1020A0002034203420342034203420342034203490
:1020B0002034003452346F347434613474346934ED
:1020C0006F346E3420344E346F3472346D34613476
:1020D0006C346534003452346F3474346134743485
:1020E00069346F346E34203449346E347634653458
:1020F00072347334653400342034413452345234F1
:1021000045345434203445344E34203443344F3431
:102110005534523453342034003454342F346D3415
:102120006E340034563465347234203431342E34F5
:1021300030342034323432342F34303436342F3487
:10214000303438340034443461346E3469346534A6
:102150006C3420344734753469346C346C346534F1
:102160006D346F346E340034FF3FFF3FFF3FFF3F5D
:10260000A8000E23003E031908008A110A12E921CE
:102610008A110A16A80A0319A70A012B27088A009B
:10262000280882008A110A12E6211030A700923091
:10263000A8008A110A1600238A110A12E02110301C
:10264000A700A330A8008A110A1600238A110A12D3
:102650000830AD006C21E621D421E021D4217A2874
:103F38008A110A124B28FF3F830183162430980008
:103F48000C309900831290309800EB27C13C031D78
:103F5800FC2F3130990083014B309900F801EB2791
:103F680003178F00FE00EB2703178D00EB27F900DE
:103F7800FA00FA0A1F308400EB27840A8000FA0B43
:103F8800C02FF808031DE82F0317203084006400B1
:103F980000088C00840A00088E00840A83168C139B
:103FA8007E1F8C170C1555308D00AA308D008C148F
:103FB800000000008C18DE2F0C1183128D0A7E1F62
:103FC800F903F90BCB2FAF2F4E309900B22F830195
:103FD8000330FB00FC01FD018C1EF52F1A08F807C1
:103FE80008006400FD0BF02FFC0BEF2FFB0BEE2FEE
:083FF80098139C2FFF3FFF3FCF
:08400000FF3FFF3FFF3FFF3FC0
:02400E00323F3F
:00000001FF
